:0A0E7100000102020303040405055A
:10069600E4F52CF52BF52AF529C203C200C202C2E5
:1006A60001120E937E0A7F008E0A8F0B75120A7551
:1006B600131275080A75091C75100A75114A751406
:1006C6000A751578EE54C0700302079B752D0075E8
:1006D6002E808E2F8F30C374AE9FFF740A9ECF2458
:1006E60002CF3400FEE48F288E27F526F525F52463
:1006F600F523F522F521AF28AE27AD26AC25AB2490
:10070600AA23A922A821C3120AFF5037E5302524BF
:10071600F582E52F3523F583E0FFE52E2524F582C6
:10072600E52D3523F583EFF0E4FAF9F8E524240105
:10073600F524EA3523F523E93522F522E83521F5B6
:100746002180B3852D0A852E0B74002480FF740A40
:1007560034FFFEC3E5139FF513E5129EF512C3E5BC
:100766000D9FF50DE50C9EF50CC3E50F9FF50FE506
:100776000E9EF50EC3E5099FF509E5089EF508C32B
:10078600E5119FF511E5109EF510C3E5159FF515CA
:10079600E5149EF514D2E843D82090E668E04409B3
:1007A600F090E65CE0443DF0D2AF90E680E054F78E
:1007B600F0538EF8C203120EA53001051203DAC2F9
:1007C600013003F21208FE50EDC203120D6C200038
:1007D6001690E682E030E704E020E1EF90E682E062
:0F07E60030E604E020E0E4120D151209FE80C792
:0107F50022E1
:100E2C0090E60AE054F0600B90E509E030E402D360
:050E3C0022C322D322B5
:1003DA0090E6B9E070030204C514700302056E24A6
:1003EA00FE700302060724FB70030204BF147003A5
:1003FA000204B91470030204AD1470030204B32496
:10040A00056003020682120E9D400302068E90E6E4
:10041A00BBE024FE603B14605624FD601614604065
:10042A0024067075E50A90E6B3F0E50B90E6B4F0A1
:10043A0002068E120E2C500FE51290E6B3F0E51369
:10044A0090E6B4F002068E90E6A0E04401F00206BF
:10045A008EE50C90E6B3F0E50D90E6B4F002068E58
:10046A00E50E90E6B3F0E50F90E6B4F002068E9042
:10047A00E6BAE0FF120D41AA06A9077B01EA494B39
:10048A00600DEE90E6B3F0EF90E6B4F002068E90BF
:10049A00E6A0E04401F002068E90E6A0E04401F0F6
:1004AA0002068E120E5302068E120E8302068E1258
:1004BA000E7B02068E120E4102068E120E9F40031A
:1004CA0002068E90E6B8E0247F602B14603C24027A
:1004DA006003020564A200E433FF25E0FFA202E400
:1004EA00334F90E740F0E4A3F090E68AF090E68B71
:1004FA007402F002068EE490E740F0A3F090E68AD8
:10050A00F090E68B7402F002068E90E6BCE0547E10
:10051A00FF7E00E0D3948040067C007D0180047C4D
:10052A00007D00EC4EFEED4F2471F582740E3EF50F
:10053A0083E493FF3395E0FEEF24A1FFEE34E68FC8
:10054A0082F583E0540190E740F0E4A3F090E68A54
:10055A00F090E68B7402F002068E90E6A0E0440169
:10056A00F002068E120EA1400302068E90E6B8E053
:10057A0024FE601D2402600302068E90E6BAE0B4EF
:10058A000105C20002068E90E6A0E04401F00206D0
:10059A008E90E6BAE0705990E6BCE0547EFF7E0089
:1005AA00E0D3948040067C007D0180047C007D00BD
:1005BA00EC4EFEED4F2471F582740E3EF583E49302
:1005CA00FF3395E0FEEF24A1FFEE34E68F82F58338
:1005DA00E054FEF090E6BCE05480FF131313541F5E
:1005EA00FFE0540F2F90E683F0E04420F002068EDD
:1005FA0090E6A0E04401F002068E02068E120EA3D7
:10060A00400302068E90E6B8E024FE6023240270BE
:10061A005E90E6BAE0B40104D200806890E6BAE0DF
:10062A00B40204805F805D90E6A0E04401F080544B
:10063A0090E6BCE0547EFF7E00E0D3948040067CC6
:10064A00007D0180047C007D00EC4EFEED4F24719C
:10065A00F582740E3EF583E493FF3395E0FEEF24B2
:10066A00A1FFEE34E68F82F583E04401F080159015
:10067A00E6A0E04401F0800C120080500790E6A04A
:0B068A00E04401F090E6A0E04480F0A6
:010695002242
:03003300020E9921
:040E990053D8EF3209
:060E9300D200120E8B22BA
:010EA500222A
:0208FE00D32203
:0209FE00D32202
:020E9D00D3225E
:080E7B0090E6BAE0F51ED32257
:100E410090E740E51EF0E490E68AF090E68B04F02E
:020E5100D322AA
:080E830090E6BAE0F51CD32251
:100E530090E740E51CF0E490E68AF090E68B04F01E
:020E6300D32298
:020E9F00D3225C
:020EA100D3225A
:020EA300D32258
:1000800090E678E05410FFC4540F4450F51D13E47B
:1000900033F51F90E6B9E0245EB40A004003020382
:1000A000D89000AF75F003A4C58325F0C583730213
:1000B000024D02024D0203D80203D80200CD020312
:1000C000D80201130201390200ED02010090E6009E
:1000D000E0FFC4540F90E740F0E490E68AF090E629
:1000E0008B04F090E6A0E04480F00203D890E67A1A
:1000F000E054FEF0E490E68AF090E68BF00203D83C
:1001000090E67AE04401F0E490E68AF090E68BF025
:100110000203D890E7407407F0E490E68AF090E696
:100120008B04F090E6A0E04480F07FE87E031209A3
:10013000B8D204120CE60203D8751F01431D0190CA
:10014000E6BAE0753100F532A3E0FEE4EE4231900C
:10015000E6BEE0753300F534A3E0FEE4EE423390F2
:10016000E6B8E064C060030201F3E5344533700390
:100170000203D890E6A0E020E1F9C3E5349440E51D
:100180003394005008853335853436800675350044
:10019000753640E4F537F538C3E5389536E53795DB
:1001A00035501874402538F582E434E7F58374CD72
:1001B000F00538E5387002053780DDAD367AE7792D
:1001C000407EE77F40AB07AF32AE31120B10E490B8
:1001D000E68AF090E68BE536F02532F532E53535E6
:1001E00031F531C3E5349536F534E5339535F533DE
:1001F00002016A90E6B8E0644060030203D8E53487
:10020000453370030203D8E490E68AF090E68BF061
:1002100090E6A0E020E1F990E68BE0753500F53638
:10022000FD7AE779407EE77F40AB07AF32AE31120F
:100230000C4BE5362532F532E5353531F531C3E580
:10024000349536F534E5339535F53380B1E4F51F53
:1002500090E6BAE0753100F532A3E0FEE4EE4231FB
:1002600090E6BEE0753300F534A3E0FEE4EE4233E1
:1002700090E6B8E064C06003020340E534453370A3
:10028000030203D890E6A0E020E1F9C3E5349440EE
:10029000E53394005008853335853436800675354E
:1002A0000075364090E6B9E0B4A335E4F537F5388B
:1002B000C3E5389536E53795355060E5322538F594
:1002C00082E5313537F583E0FF74402538F582E467
:1002D00034E7F583EFF00538E5387002053780D054
:1002E000E4F537F538C3E5389536E53795355018D8
:1002F00074402538F582E434E7F58374CDF0053891
:10030000E5387002053780DDAD367AE779407EE763
:100310007F40AB07AF32AE31120B10E490E68AF0AB
:1003200090E68BE536F02532F532E5353531F5319D
:10033000C3E5349536F534E5339535F53302027B64
:1003400090E6B8E0644060030203D8E534453370BA
:10035000030203D8E490E68AF090E68BF090E6A0E2
:10036000E020E1F990E68BE0753500F53690E6B9CE
:10037000E0B4A335E4F537F538C3E5389536E5370D
:100380009535503874402538F582E434E7F583E03C
:10039000FFE5322538F582E5313537F583EFF00595
:1003A00038E5387002053780D0AD367AE779407E7F
:1003B000E77F40AB07AF32AE31120C4BE53625324A
:1003C000F532E5353531F531C3E5349536F534E5AB
:0903D000339535F53302034BC3EC
:0103D9002201
:100D9100C0E0C083C08290E6B5E04401F0D20153C7
:0F0DA10091EF90E65D7401F0D082D083D0E03204
:100E0000C0E0C083C0825391EF90E65D7404F0D0DF
:060E100082D083D0E03225
:100E1600C0E0C083C0825391EF90E65D7402F0D0CB
:060E260082D083D0E0320F
:100BDD00C0E0C083C08290E680E030E70E85080C4F
:100BED0085090D85100E85110F800C85100C851152
:100BFD000D85080E85090F5391EF90E65D7410F089
:070C0D00D082D083D0E03259
:100DE800C0E0C083C082D2035391EF90E65D7408DF
:080DF800F0D082D083D0E0327C
:100C1400C0E0C083C08290E680E030E70E85080C17
:100C240085090D85100E85110F800C85100C85111A
:100C34000D85080E85090F5391EF90E65D7420F041
:070C4400D082D083D0E03222
:010EA6003219
:010EA7003218
:010EA8003217
:010EA9003216
:010EAA003215
:010EAB003214
:010EAC003213
:010EAD003212
:010EAE003211
:010EAF003210
:010EB000320F
:010EB100320E
:010EB200320D
:010EB300320C
:010EB400320B
:010EB500320A
:010EB6003209
:010EB7003208
:010EB8003207
:010EB9003206
:010EBA003205
:010EBB003204
:010EBC003203
:010EBD003202
:010EBE003201
:010EBF003200
:010EC00032FF
:010EC10032FE
:010EC20032FD
:010EC30032FC
:010EC40032FB
:010EC50032FA
:010EC60032F9
:010EC70032F8
:010EC80032F7
:010EC90032F6
:060B5B00AB07AA06AC0581
:100B6100E4FDE51F6010EA7E000DEE2400F582E44D
:100B71003410F583EAF0EBAE050D74002EF582E436
:100B81003410F583EBF0AF050D74002FF582E434DA
:100B910010F583ECF07A107B00AF1D120DCCAF1D68
:030BA100120BA58F
:010BA400222E
:0A0C4B008E398F3A8D3B8A3C8B3DB9
:100C5500E4F53EE53EC3953B5020053AE53AAE390D
:100C65007002053914FFE53D253EF582E4353CF576
:0A0C750083E0FD120B5B053E80D901
:010C7F002252
:0A0B10008E398F3A8D3B8A3C8B3DF5
:100B1A00E4FDF53EE51F6012E539FF7E000DEE2487
:100B2A0000F582E43410F583EFF0E53AAE050D7472
:100B3A00002EF582E43410F583E53AF07A107B0052
:100B4A00AF1D120DCCAB3DAA3CAD3BAF1D120DB093
:010B5A002278
:100A000012010002000000400516408100000102B2
:100A100000010A06000200000040010009022E0049
:100A200001010080320904000004FF0000000705F6
:100A30000202000200070504020002000705860208
:100A40000002000705880200020009022E000101D1
:100A50000080320904000004FF00000007050202C4
:100A60004000000705040240000007058602400020
:100A70000007058802400000040309040C0341003C
:100A80004300430045005300260355005300420035
:100A90002D00410049004F00310036002D0031008B
:100AA00036004100000000000000000000000000CF
:03004300020900AF
:030053000209009F
:10090000020D9100020E1600020E0000020DE8001A
:10091000020BDD00020C1400020EA600020EA7005E
:10092000020EA800020EA900020EAA00020EAB00E1
:10093000020EAC00020EAD00020EAE00020EAF00C1
:10094000020EB000020EA700020EB100020EB200AD
:10095000020EB300020EB400020EB500020EB60085
:10096000020EB700020EA700020EA700020EA7009B
:10097000020EB800020EB900020EBA00020EBB0051
:10098000020EBC00020EBD00020EBE00020EBF0031
:10099000020EC000020EC100020EC200020EC30011
:1009A000020EC400020EC500020EC600020EC700F1
:0809B000020EC800020EC9008E
:100D150090E682E030E004E020E60B90E682E030E9
:100D2500E119E030E71590E680E04401F07F147E9C
:0C0D3500001209B890E680E054FEF022A5
:100CE60030040990E680E0440AF0800790E680E050
:100CF6004408F07FDC7E051209B890E65D74FFF0CB
:0F0D060090E65FF05391EF90E680E054F7F02213
:1009B8008E398F3A90E600E054187012E53A240117
:1009C800FFE43539C313F539EF13F53A801590E68E
:1009D80000E05418FFBF100BE53A25E0F53AE53979
:1009E80033F539E53A153AAE39700215394E6005D6
:0609F800120D8080EE22CA
:080E8B00E4F51BD2E9D2AF220D
:100BA500AD0790E678E020E6F9C2E990E678E04402
:100BB50080F0ED25E090E679F090E678E030E0F918
:100BC50090E678E04440F090E678E020E6F990E69B
:080BD50078E030E1D6D2E922FC
:100CB400AC0790E678E020E6F9E51B702390E6782F
:100CC400E04480F0EC25E090E679F08D16AF03A9BE
:100CD400077517018A188919E4F51A751B01D322BF
:020CE400C32229
:100C8000AC0790E678E020E6F9E51B702590E67861
:100C9000E04480F0EC25E0440190E679F08D16AF59
:100CA00003A9077517018A188919E4F51A751B033A
:040CB000D322C32266
:03004B000207F6B3
:1007F600C0E0C083C082C085C084C086758600C044
:10080600D075D000C000C001C002C003C006C0073A
:1008160090E678E030E206751B060208E090E6787E
:10082600E020E10CE51B64026006751B070208E088
:10083600E51B24FE605F14603624FE70030208D1B7
:1008460024FC70030208DD240860030208E0AB17ED
:10085600AA18A919AF1A051A8F82758300120AB051
:1008660090E679F0E51A65167070751B05806B9039
:10087600E679E0AB17AA18A919AE1A8E827583001D
:10088600120ADD751B02E5166401704E90E678E0EB
:100896004420F08045E51624FEB51A0790E678E078
:1008A6004420F0E51614B51A0A90E678E04440F0C4
:1008B600751B0090E679E0AB17AA18A919AE1A8E37
:1008C60082758300120ADD051A800F90E678E044EF
:1008D60040F0751B008003751B005391DFD007D0D5
:1008E60006D003D002D001D000D0D0D086D084D09C
:0808F60085D082D083D0E032EE
:020D4100A90700
:100D4300AE14AF158F828E83A3E064037017AD01D9
:100D530019ED7001228F828E83E07C002FFDEC3E23
:080D6300FEAF0580DFE4FEFF96
:010D6B002265
:100DB000120C80E51B24FA600E146006240770F301
:0C0DC000D322E4F51BD322E4F51BD32260
:100DCC00120CB4E51B24FA600E146006240770F3B1
:0C0DDC00D322E4F51BD322E4F51BD32244
:100D6C0090E682E044C0F090E681F04387010000F9
:040D7C000000002251
:100D80007400F58690FDA57C05A3E582458370F986
:010D90002240
:03000000020E6588
:0C0E6500787FE4F6D8FD75813E02069609
:100AB000BB010CE58229F582E5833AF583E02250FB
:100AC00006E92582F8E622BBFE06E92582F8E22245
:0D0AD000E58229F582E5833AF583E493225F
:100ADD00F8BB010DE58229F582E5833AF583E8F04F
:100AED00225006E92582C8F622BBFE05E92582C8FB
:020AFD00F222E3
:100AFF00EB9FF5F0EA9E42F0E99D42F0E89C45F04D
:010B0F0022C3
:00000001FF
